:10000000000000308A00412803178D0083168C13EE
:100010000C1483120C083C2803178C0083168C13D5
:100020000C1555308D00AA308D008C148C181628B4
:100030000C113C28A501A400FF30A407031CA50750
:10004000031C3C280330A300DF3028201C28A30118
:10005000E83EA200A309FC30031C3128A2070318C4
:100060002E28A2070000A30F2E2822183728A21C32
:100070003B2800003B280800831383120313000071
:1000800008000130A500F4308A011B208316850189
:100090003F3086008701880183128A110A164920A1
:1000A0000130A500F4308A011B20803087003230F7
:1000B0008A010420C7003C308A010420C80087015F
:1000C0008A110A12061967288A150A126F2A8A11DC
:1000D0000A12061C6E288A150A12682EA101A001B8
:1000E0008A110A12D62A003021078A007E302007A2
:1000F00003188A0AA00A0319A10A820001340034F5
:10010000003400340034003400340034003400344F
:10011000023400340034003400340034003400343D
:10012000003400340434003400340034003400342B
:100130000034003400340034083400340034003417
:1001400000340034003400340034003410340034FF
:1001500000340034003400340034003400340034FF
:1001600020340034003400340034003400340034CF
:1001700000340034003401340034003400340034DE
:1001800000340034003400340034023400340034CD
:1001900000340034003400340034003400340434BB
:1001A00000340034003400340034003400340034AF
:1001B0000034083400340034003400340034003497
:1001C000003400340034103400340034003400347F
:1001D000003400340034003400342034003400345F
:1001E000003400340034003400340034003400346F
:1001F000013400340034003400340034003400345E
:10020000003400340234003400340034003400344C
:10021000003400340034003404340034003400343A
:100220000034003400340034003400340834003426
:10023000003400340034003400340034003400341E
:1002400010340034003400340034003400340034FE
:1002500000340034203400340034003400340034DE
:1002600000340034003400340034013400340034ED
:1002700000340034003400340034003400340234DC
:1002800000340034003400340034003400340034CE
:1002900000340434003400340034003400340034BA
:1002A00000340034003408340034003400340034A6
:1002B000003400340034003400341034003400348E
:1002C000003400340034003400340034003420346E
:1002D000003400340034003400340034003400347E
:1002E000003400340134003400340034003400346D
:1002F000003400340034003402340034003400345C
:100300000034003400340034003400340434003449
:10031000003400340034003400340034003400343D
:100320000834003400340034003400340034003425
:10033000003400341034003400340034003400340D
:1003400000340034003400342034003400340034ED
:1003500000340034003400340034003400340134FC
:1003600000340034003400340034003400340034ED
:1003700000340234003400340034003400340034DB
:1003800000340034003404340034003400340034C9
:1003900000340034003400340034083400340034B5
:1003A000003400340034003400340034003410349D
:1003B000003400340034003400340034003400349D
:1003C000003420340034003400340034003400346D
:1003D000003400340034003401340034003400347C
:1003E000003400340034003400340034023400346B
:1003F000003400340034003400340034003400345D
:100400000434003400340034003400340034003448
:100410000034003408340034003400340034003434
:10042000003400340034003410340034003400341C
:1004300000340034003400340034003420340034FC
:10044000003400340034003400340034003400340C
:1004500000340134003400340034003400340034FB
:1004600000340034003402340034003400340034EA
:1004700000340034003400340034043400340034D8
:1004800000340034003400340034003400340834C4
:1004900000340034003400340034003400340034BC
:1004A000003410340034003400340034003400349C
:1004B000003400340034203400340034003400347C
:1004C000003400340034003400340034013400348B
:1004D000003400340034003400340034003400347C
:1004E000023400340034003400340034003400346A
:1004F0000034003404340034003400340034003458
:100500000034003400340034083400340034003443
:10051000003400340034003400340034103400342B
:10052000003400340034003400340034003400342B
:1005300020340034003400340034003400340034FB
:10054000003400340034013400340034003400340A
:1005500000340034003400340034023400340034F9
:1005600000340034003400340034003400340434E7
:1005700000340034003400340034003400340034DB
:1005800000340834003400340034003400340034C3
:1005900000340034003410340034003400340034AB
:1005A00000340034003400340034203487018801E2
:1005B000C6013C3030028A110A12031DE22A8A1158
:1005C0000A12752FB00A8A017320A6008A017320CF
:1005D000A7008A017320A8008A017320A9008A015C
:1005E0007320AA008A017320AB008A017320AC003B
:1005F0008A017320AD008A017320AE008A01732046
:10060000AF008A110A12061C082B8A150A12682EDE
:100610008A110A1206190F2B8A150A126F2A8A11DB
:100620000A128619162B8A110A12752F8A110A12BC
:10063000861C1D2B8A110A12452D083033028A119F
:100640000A12031D262B8A110A12532C013036027E
:100650008A110A12031D2F2B8A110A128F2C0830BF
:1006600038028A110A12031D382B8A110A12CA2C69
:10067000013031028A110A12031D412B8A110A121C
:10068000042D0130850047088A0127200130260209
:100690008A110A12031D4E2B0230850020302602DB
:1006A0008A110A12031D562B0230850010302702D2
:1006B0008A110A12031D5E2B0230850008302802C1
:1006C0008A110A12031D662B0230850004302902AC
:1006D0008A110A12031D6E2B0230850002302A0295
:1006E0008A110A12031D762B0230850001302B027D
:1006F0008A110A12031D7E2B0230850020302B0246
:100700008A110A12031D862B0230850010302C023C
:100710008A110A12031D8E2B0230850008302D022B
:100720008A110A12031D962B0230850004302E0216
:100730008A110A12031D9E2B0230850002302F02FF
:100740008A110A12031DA62B02308500C60A310841
:1007500087003B0888001930A30091308A012820C7
:10076000260887002608880003308A011A204030B6
:100770008700320887003C08880007308A011A2069
:10078000270887002708880003308A011A20403094
:100790008700330887003D08880007308A011A2047
:1007A000280887002808880003308A011A20403072
:1007B0008700340887003E08880007308A011A2025
:1007C000290887002908880003308A011A20403050
:1007D0008700350887003F08880007308A011A2003
:1007E0002A0887002A08880003308A011A2040302E
:1007F0008700360887004008880007308A011A20E1
:100800002B0887002B08880003308A011A2040300B
:100810008700370887004108880007308A011A20BE
:100820002C0887002C08880003308A011A204030E9
:100830008700380887004208880007308A011A209C
:100840002D0887002D08880003308A011A204030C7
:100850008700390887004308880007308A011A207A
:100860002E0887002E08880003308A011A204030A5
:1008700087003A0887004408880007308A011A2058
:100880002F0887002F08880003308A011A20403083
:100890008700323046028A110A12031D512C8A0148
:1008A000D62A8A01A62B26088A110A12031D5A2C61
:1008B00002308500013026028A110A12031D622CC3
:1008C00006308500023026028A110A12031D6A2CA6
:1008D00001308500043026028A110A12031D722C91
:1008E00002308500083026028A110A12031D7A2C74
:1008F00002308500103026028A110A12031D822C54
:1009000002308500203026028A110A12031D8A2C2B
:10091000023085000000000000008A01A62B260896
:100920008A110A12031D962C02308500013026021E
:100930008A110A12031D9E2C063085000230260201
:100940008A110A12031DA62C0130850004302602EC
:100950008A110A12031DAE2C0630850008302602CB
:100960008A110A12031DB62C0130850010302602B0
:100970008A110A12031DBE2C023085002030260287
:100980008A110A12031DC62C0230850000000000E7
:100990008A01A62B26088A110A12031DD12C0230C7
:1009A0008500013026028A110A12031DD92C063057
:1009B0008500023026028A110A12031DE12C013043
:1009C0008500043026028A110A12031DE92C063024
:1009D0008500083026028A110A12031DF12C01300D
:1009E0008500103026028A110A12031DF92C0630E8
:1009F0008500203026028A110A12031D012D0130C4
:100A0000850000008A01A62B26088A110A12031D00
:100A10000B2D02308500013026028A110A12031DB7
:100A2000132D06308500023026028A110A12031D9A
:100A30001B2D01308500043026028A110A12031D85
:100A4000232D06308500083026028A110A12031D64
:100A50002B2D05308500103026028A110A12031D45
:100A6000332D06308500203026028A110A12031D1C
:100A70003B2D05308500013027028A110A12031D23
:100A8000432D013085008A01A62B083033028A11DC
:100A90000A12031D4E2D8A110A127B2E01303602D6
:100AA0008A110A12031D572D8A110A12B72E083017
:100AB00038028A110A12031D602D8A110A12F22EC1
:100AC000013031028A110A12031D692D8A110A129E
:100AD0002C2F48088A012720023085000130260289
:100AE0008A110A12031D762D01308500203026025E
:100AF0008A110A12031D7E2D013085001030270255
:100B00008A110A12031D862D013085000830280243
:100B10008A110A12031D8E2D01308500043029022E
:100B20008A110A12031D962D0130850002302A0217
:100B30008A110A12031D9E2D0130850001302B02FF
:100B40008A110A12031DA62D0130850020302B02C8
:100B50008A110A12031DAE2D0130850010302C02BF
:100B60008A110A12031DB62D0130850008302D02AE
:100B70008A110A12031DBE2D0130850004302E0299
:100B80008A110A12031DC62D0130850002302F0282
:100B90008A110A12031DCE2D01308500C60A3108C4
:100BA00087003B0888001930A30091308A01282073
:100BB000260887002608880003308A011A20403062
:100BC0008700320887003C08880007308A011A2015
:100BD000270887002708880003308A011A20403040
:100BE0008700330887003D08880007308A011A20F3
:100BF000280887002808880003308A011A2040301E
:100C00008700340887003E08880007308A011A20D0
:100C1000290887002908880003308A011A204030FB
:100C20008700350887003F08880007308A011A20AE
:100C30002A0887002A08880003308A011A204030D9
:100C40008700360887004008880007308A011A208C
:100C50002B0887002B08880003308A011A204030B7
:100C60008700370887004108880007308A011A206A
:100C70002C0887002C08880003308A011A20403095
:100C80008700380887004208880007308A011A2048
:100C90002D0887002D08880003308A011A20403073
:100CA0008700390887004308880007308A011A2026
:100CB0002E0887002E08880003308A011A20403051
:100CC00087003A0887004408880007308A011A2004
:100CD0002F0887002F08880003308A011A2040302F
:100CE0008700323046028A110A12031D792E8A01CA
:100CF000D62A8A01CE2D26088A110A12031D822EB9
:100D000001308500013026028A110A12031D8A2E45
:100D100001308500023026028A110A12031D922E2C
:100D200002308500043026028A110A12031D9A2E11
:100D300001308500083026028A110A12031DA22EF6
:100D400001308500103026028A110A12031DAA2ED6
:100D500001308500203026028A110A12031DB22EAE
:100D6000013085000000000000008A01CE2D260819
:100D70008A110A12031DBE2E0130850001302602A1
:100D80008A110A12031DC62E013085000230260288
:100D90008A110A12031DCE2E02308500043026026D
:100DA0008A110A12031DD62E013085000830260252
:100DB0008A110A12031DDE2E023085001030260231
:100DC0008A110A12031DE62E01308500203026020A
:100DD0008A110A12031DEE2E01308500000000006A
:100DE0008A01CE2D26088A110A12031DF92E013020
:100DF0008500013026028A110A12031D012F0130DD
:100E00008500023026028A110A12031D092F0230C2
:100E10008500043026028A110A12031D112F0130A9
:100E20008500083026028A110A12031D192F02308C
:100E30008500103026028A110A12031D212F01306D
:100E40008500203026028A110A12031D292F023044
:100E5000850000008A01CE2D26088A110A12031D82
:100E6000332F01308500013026028A110A12031D3A
:100E70003B2F01308500023026028A110A12031D21
:100E8000432F02308500043026028A110A12031D06
:100E90004B2F01308500083026028A110A12031DEB
:100EA000532F02308500103026028A110A12031DCA
:100EB0005B2F01308500203026028A110A12031DA3
:100EC000632F02308500013027028A110A12031DA8
:100ED0006B2F01308500023027028A110A12031D90
:100EE000732F023085008A01CE2DB001A101A0012F
:100EF0000310B10D403031028A110A12031D832FF5
:100F00008A110A12EF2F0310B20D403032028A11FB
:100F10000A12031D8E2F8A150A128E280310B30D94
:100F2000403033028A110A12031D992F8A110A12C6
:100F3000EF2F0310B40D403034028A110A12031D42
:100F4000A42F8A150A128E280310B50D40303502E1
:100F50008A110A12031DAF2F8A110A12EF2F0310F4
:100F6000B60D403036028A110A12031DBA2F8A15B7
:100F70000A128E280310B70D403037028A110A1268
:100F8000031DC52F8A110A12EF2F0310B80D403030
:100F900038028A110A12031DD02F8A150A128E28D0
:100FA0000310B90D403039028A110A12031DDB2FDC
:100FB0008A110A12EF2F0310BA0D40303A028A113B
:100FC0000A12031DE62F8A150A128E288A110A12A8
:100FD0008619ED2F8A150A12A5298A01D62A4030D2
:100FE00031028A110A12031DF72F0130B20040307E
:100FF00031028A110A12031DFE2FB1014030320264
:101000008A150A12031D06280130B300403032024F
:101010008A150A12031D0D28B201403033028A15C9
:101020000A12031D15280130B400403033028A151E
:101030000A12031D1C28B301403034028A150A121B
:10104000031D24280130B500403034028A150A12ED
:10105000031D2B28B401403035028A150A12031DE6
:1010600033280130B600403035028A150A12031DBC
:101070003A28B501403036028A150A12031D42286B
:101080000130B700403036028A150A12031D492884
:10109000B601403037028A150A12031D512801306B
:1010A000B800403037028A150A12031D5828B701CC
:1010B000403038028A150A12031D60280130B90039
:1010C000403038028A150A12031D6728B8014030E3
:1010D00039028A150A12031D6F280130BA00403008
:1010E00039028A150A12031D7628B90140303A02E6
:1010F0008A150A12031D7E280130B10040303A02E1
:101100008A150A12031D8528BA018A150A12861942
:101110008C288A150A12A5298A01D62A0310BB0D2C
:1011200040303B028A150A12031D99288A150A12BB
:10113000FE280310BC0D40303C028A150A12031D24
:10114000A4288A150A12FE280310BD0D40303D0266
:101150008A150A12031DAF288A150A12FE280310E9
:10116000BE0D40303E028A150A12031DBA288A15A8
:101170000A12FE280310BF0D40303F028A150A12E2
:10118000031DC5288A150A12FE280310C00D403021
:1011900040028A150A12031DD0288A150A12FE2859
:1011A0000310C10D403041028A150A12031DDB28CD
:1011B0008A150A12FE280310C20D403042028A1519
:1011C0000A12031DE6288A150A12FE280310C30D11
:1011D000403043028A150A12031DF1288A150A12AB
:1011E000FE280310C40D403044028A150A12031D64
:1011F000FC288A150A12FE288A01EF2F40303B0294
:101200008A150A12031D06290130BC0040303B023A
:101210008A150A12031D0D29BB0140303C028A15B4
:101220000A12031D15290130BD0040303C028A1509
:101230000A12031D1C29BC0140303D028A150A1206
:10124000031D24290130BE0040303D028A150A12D8
:10125000031D2B29BD0140303E028A150A12031DD1
:1012600033290130BF0040303E028A150A12031DA7
:101270003A29BE0140303E028A150A12031D422956
:101280000130BF0040303E028A150A12031D492971
:10129000BE0140303F028A150A12031D5129013058
:1012A000C00040303F028A150A12031D5829BF01B1
:1012B000403040028A150A12031D60290130C10026
:1012C000403040028A150A12031D6729C0014030D0
:1012D00041028A150A12031D6F290130C2004030F5
:1012E00041028A150A12031D7629C10140304202CB
:1012F0008A150A12031D7E290130C30040304202C4
:101300008A150A12031D8529C201403043028A153D
:101310000A12031D8D290130C400403043028A1592
:101320000A12031D9429C301403044028A150A128F
:10133000031D9C290130BB00403044028A150A126B
:10134000031DA329C4018A01EF2F8A017320A6007F
:101350008A017320A7008A017320A8008A017320E4
:10136000A9008A017320AA008A017320AB008A01B8
:101370007320AC008A017320AD008A017320AE0097
:101380008A017320AF00310887003B0888001930BC
:10139000A30091308A0128202608870026088800AB
:1013A00003308A011A2040308700320887003C0849
:1013B000880007308A011A2027088700270888003C
:1013C00003308A011A2040308700330887003D0827
:1013D000880007308A011A2028088700280888001A
:1013E00003308A011A2040308700340887003E0805
:1013F000880007308A011A202908870029088800F8
:1014000003308A011A2040308700350887003F08E2
:10141000880007308A011A202A0887002A088800D5
:1014200003308A011A2040308700360887004008C0
:10143000880007308A011A202B0887002B088800B3
:1014400003308A011A20403087003708870041089E
:10145000880007308A011A202C0887002C08880091
:1014600003308A011A20403087003808870042087C
:10147000880007308A011A202D0887002D0888006F
:1014800003308A011A20403087003908870043085A
:10149000880007308A011A202E0887002E0888004D
:1014A00003308A011A20403087003A088700440838
:1014B000880007308A011A202F0887002F0888002B
:1014C00003308A011A20403087008A150A128619D3
:1014D0006C2A8A150A12C329C6018A01012B8501CB
:1014E00005150530A500DC308A011B2085018A1511
:1014F0000A12861C7E2A8A110A167B28B001C601B0
:10150000A101A001310887003B08880005308A014D
:101510001A2040308700320887003C0888000530D8
:101520008A011A2040308700330887003D08880070
:1015300005308A011A2040308700340887003E08B1
:10154000880005308A011A2040308700350887005E
:101550003F08880005308A011A204030870036088D
:1015600087004008880005308A011A204030870033
:10157000370887004108880005308A011A2040306A
:101580008700380887004208880005308A011A2041
:1015900040308700390887004308880005308A01F9
:1015A0001A20403087003A08870044088800053038
:1015B0008A011A20803087008701880185018A15F9
:1015C0000A12861AE62A8A150A120E2B8A150A12A0
:1015D000061AED2A8A150A123D2D8A150A12861955
:1015E000F42A8A110A1649208A150A12061DF92AB8
:1015F00087018A150A12061DFF2A013085008A1507
:101600000A12061D052B8A0155288A150A12061C86
:101610000B2B8A0155288A150A12772A0130A5005A
:10162000F4308A011B208A150A12861A1A2B8A1591
:101630000A120E2B0310B10D403031028A150A1226
:10164000031D252B8A150A128B2B0310B20D403077
:1016500032028A150A12031D302B8A150A12242C15
:101660000310B30D403033028A150A12031D3B2BC1
:101670008A150A128B2B0310B40D403034028A15E0
:101680000A12031D462B8A150A12242C0310B50DCD
:10169000403035028A150A12031D512B8A150A1291
:1016A0008B2B0310B60D403036028A150A12031D2B
:1016B0005C2B8A150A12242C0310B70D4030370218
:1016C0008A150A12031D672B8A150A128B2B031029
:1016D000B80D403038028A150A12031D722B8A1584
:1016E0000A12242C0310B90D403039028A150A124F
:1016F000031D7D2B8A150A128B2B0310BA0D403067
:101700003A028A150A12031D882B8A150A12242C04
:101710008A150A12772A403031028A150A12031DEF
:10172000932B0130B200403031028A150A12031D9A
:101730009A2BB101403032028A150A12031DA22BE6
:101740000130B300403032028A150A12031DA92B62
:10175000B201403033028A150A12031DB12B013049
:10176000B400403033028A150A12031DB82BB301AE
:10177000403034028A150A12031DC02B0130B50017
:10178000403034028A150A12031DC72BB4014030C1
:1017900035028A150A12031DCF2B0130B6004030E6
:1017A00035028A150A12031DD62BB50140303602C8
:1017B0008A150A12031DDE2B0130B70040303602B5
:1017C0008A150A12031DE52BB601403037028A152F
:1017D0000A12031DED2B0130B800403037028A1584
:1017E0000A12031DF42BB701403038028A150A1281
:1017F000031DFC2B0130B900403038028A150A1253
:10180000031D032CB801403039028A150A12031D4A
:101810000B2C0130BA00403039028A150A12031D20
:10182000122CB90140303A028A150A12031D1A2CF3
:101830000130B10040303A028A150A12031D212CF2
:10184000BA018A150A12772A0310BB0D40303B02F9
:101850008A150A12031D2F2C8A150A12952C0310C3
:10186000BC0D40303C028A150A12031D3A2C8A1521
:101870000A12952C0310BD0D40303D028A150A1244
:10188000031D452C8A150A12952C0310BE0D4030FD
:101890003E028A150A12031D502C8A150A12952C35
:1018A0000310BF0D40303F028A150A12031D5B2C46
:1018B0008A150A12952C0310C00D403040028A157B
:1018C0000A12031D662C8A150A12952C0310C10DED
:1018D000403041028A150A12031D712C8A150A1222
:1018E000952C0310C20D403042028A150A12031DC6
:1018F0007C2C8A150A12952C0310C30D403043022C
:101900008A150A12031D872C8A150A12952C0310BA
:10191000C40D403044028A150A12031D922C8A1508
:101920000A12952C8A150A128B2B40303B028A151D
:101930000A12031D9D2C0130BC0040303B028A1569
:101940000A12031DA42CBB0140303C028A150A1266
:10195000031DAC2C0130BD0040303C028A150A1238
:10196000031DB32CBC0140303D028A150A12031D31
:10197000BB2C0130BE0040303D028A150A12031D07
:10198000C22CBD0140303E028A150A12031DCA2C2A
:101990000130BF0040303E028A150A12031DD12CCF
:1019A000BE0140303E028A150A12031DD92C0130B7
:1019B000BF0040303E028A150A12031DE02CBE0112
:1019C00040303F028A150A12031DE82C0130C00086
:1019D00040303F028A150A12031DEF2CBF01403030
:1019E00040028A150A12031DF72C0130C100403055
:1019F00040028A150A12031DFE2CC001403041022C
:101A00008A150A12031D062D0130C2004030410222
:101A10008A150A12031D0D2DC101403042028A159C
:101A20000A12031D152D0130C300403042028A15F1
:101A30000A12031D1C2DC201403043028A150A12EE
:101A4000031D242D0130C400403043028A150A12C0
:101A5000031D2B2DC301403044028A150A12031DB9
:101A6000332D0130BB00403044028A150A12031D99
:101A70003A2DC4018A150A128B2BC6010130A5002C
:101A8000F4308A011B208A150A12061A4A2D8A157B
:101A90000A123D2DBB01BC01BD01BE01BF01C00149
:101AA000C101C201C301C401C50A183045028A152B
:101AB0000A12031D5D2D0C30C5000C3045028A153D
:101AC0000A12031D652D0130BB000D3045028A1539
:101AD0000A12031D6D2D2030BB000E3045028A1501
:101AE0000A12031D752D1030BC000F3045028A15F7
:101AF0000A12031D7D2D0830BD00103045028A15E5
:101B00000A12031D852D0430BE00113045028A15CE
:101B10000A12031D8D2D0230BF00123045028A15B6
:101B20000A12031D952D0130C000133045028A159D
:101B30000A12031D9D2D2030C000143045028A1565
:101B40000A12031DA52D1030C100153045028A155B
:101B50000A12031DAD2D0830C200163045028A1549
:101B60000A12031DB52D0430C300173045028A1533
:101B70000A12031DBD2D0230C4008A150A12772AED
:101B800040303B028A150A12031DC82D0130BC00EB
:101B900040303B028A150A12031DCF2DBB01403095
:101BA0003C028A150A12031DD72D0130BD004030BA
:101BB0003C028A150A12031DDE2DBC0140303D0295
:101BC0008A150A12031DE62D0130BE0040303D0289
:101BD0008A150A12031DED2DBD0140303E028A1503
:101BE0000A12031DF52D0130BF0040303E028A1558
:101BF0000A12031DFC2DBE0140303E028A150A1256
:101C0000031D042E0130BF0040303E028A150A1227
:101C1000031D0B2EBE0140303F028A150A12031D20
:101C2000132E0130C00040303F028A150A12031DF6
:101C30001A2EBF01403040028A150A12031D222EBF
:101C40000130C100403040028A150A12031D292EBE
:101C5000C001403041028A150A12031D312E0130A5
:101C6000C200403041028A150A12031D382EC101FC
:101C7000403042028A150A12031D402E0130C30073
:101C8000403042028A150A12031D472EC20140301D
:101C900043028A150A12031D4F2E0130C400403042
:101CA00043028A150A12031D562EC3014030440216
:101CB0008A150A12031D5E2E0130BB00403044021B
:101CC0008A150A12031D652EC4018A150A12772A85
:101CD000083033028A150A12031D712E8A150A1262
:101CE0006A2F013036028A150A12031D7A2E8A15D0
:101CF0000A12A02F083038028A150A12031D832EFB
:101D00008A150A12D52F013031028A150A12031DD5
:101D10008C2E8A110A16082848088A012720850176
:101D2000013026028A150A12031D972E85012030E4
:101D300026028A150A12031D9E2E850110302702E5
:101D40008A150A12031DA52E8501083028028A155E
:101D50000A12031DAC2E8501043029028A150A12CD
:101D6000031DB32E850102302A028A150A12031DB3
:101D7000BA2E850101302B028A150A12031DC12ECD
:101D8000850120302B028A150A12031DC82E8501F9
:101D900010302C028A150A12031DCF2E850108303F
:101DA0002D028A150A12031DD62E850104302E023B
:101DB0008A150A12031DDD2E850102302F028A15B5
:101DC0000A12031DE42E8501C60A87018801193015
:101DD000A30091308A0128208701880103308A01FD
:101DE0001A20403087008701880107308A011A20B5
:101DF0008701880103308A011A204030870087015B
:101E0000880107308A011A208701880103308A017E
:101E10001A20403087008701880107308A011A2084
:101E20008701880103308A011A204030870087012A
:101E3000880107308A011A208701880103308A014E
:101E40001A20403087008701880107308A011A2054
:101E50008701880103308A011A20403087008701FA
:101E6000880107308A011A208701880103308A011E
:101E70001A20403087008701880107308A011A2024
:101E80008701880103308A011A20403087008701CA
:101E9000880107308A011A208701880103308A01EE
:101EA0001A20403087008701880107308A011A20F4
:101EB0008701880103308A011A20403087003230C0
:101EC00046028A150A12031D672F8A01D62A8A152F
:101ED0000A12E42E26088A150A12031D702F8501A6
:101EE000013026028A150A12031D772F8501023060
:101EF00026028A150A12031D7E2F85010430260250
:101F00008A150A12031D852F8501083026028A15BD
:101F10000A12031D8C2F8501103026028A150A1221
:101F2000031D932F8501203026028A150A12031DF6
:101F30009A2F85010000000000008A150A12E42E85
:101F400026088A150A12031DA62F850101302602D4
:101F50008A150A12031DAD2F8501023026028A154B
:101F60000A12031DB42F8501043026028A150A12B5
:101F7000031DBB2F8501083026028A150A12031D96
:101F8000C22F8501103026028A150A12031DC92F9F
:101F90008501203026028A150A12031DD02F8501E3
:101FA000000000008A150A12E42E26088A150A127B
:101FB000031DDB2F8501013026028A150A12031D3D
:101FC000E22F8501023026028A150A12031DE92F2D
:101FD0008501043026028A150A12031DF02F85019F
:101FE000083026028A150A12031DF72F85011030CA
:101FF00026028A150A12031DFE2F850120302602B3
:102000008A110A16031D0528850100008A01CE2DBC
:1020100026088A110A16031D0E28850101302602A2
:102020008A110A16031D15288501023026028A111D
:102030000A16031D1C288501043026028A110A167F
:10204000031D23288501083026028A110A16031D64
:102050002A288501103026028A110A16031D31280C
:102060008501203026028A110A16031D38288501B1
:10207000013027028A110A16031D3F28850102300C
:1020800027028A110A16031D462885018A150A129D
:10209000E42E05150330A500E8308A011B20051148
:1020A0000130A500F4308A011B2005150330A5007E
:1020B000E8308A011B2085010130B100B201B30173
:1020C000B401B501B601B701B801B901BA010130D7
:1020D000BB00BC01BD01BE01BF01C001C101C20105
:1020E000C301C401B0010C30C500C6010130850038
:1020F0008701880108008A110A16861882288A1525
:102100000A126F2AB001C601A101A0018A110A16A4
:1021100086198D288A110A16A52B47088A110A16D6
:10212000031D9328C901013047028A110A16031DB5
:102130009B280130C900023047028A110A16031D8C
:10214000A3280330C900033047028A110A16031D71
:10215000AB280730C900043047028A110A16031D54
:10216000B3280F30C900053047028A110A16031D33
:10217000BB281F30C900063047028A110A16031D0A
:10218000C3283F30C900073047028A110A16031CD2
:10219000CB283F30C900073047028A110A160318BE
:1021A000D228CA01073047028A110A16031DDA280D
:1021B0000130CA00083047028A110A16031DE228BE
:1021C0000330CA000A3047028A110A16031DEA28A2
:1021D0000F30CA000B3047028A110A16031DF2287D
:1021E0001F30CA000C3047028A110A16031DFA2854
:1021F0003F30CA000D3047028A110A16031C02291B
:102200003F30CA000D3047028A110A160318092907
:10221000CB010D3047028A110A16031D1129013026
:10222000CB000E3047028A110A16031D192903300C
:10223000CB000F3047028A110A16031D21290730EF
:10224000CB00103047028A110A16031D29290F30CE
:10225000CB00113047028A110A16031D31291F30A5
:10226000CB00123047028A110A16031D39293F306C
:10227000CB00133047028A110A16031C41293F3054
:10228000CB00133047028A110A1603184829CC01E3
:10229000133047028A110A16031D50290130CC0061
:1022A000143047028A110A16031D58290330CC0046
:1022B000153047028A110A16031D60290730CC0029
:1022C000163047028A110A16031D68290F30CC0008
:1022D000173047028A110A16031D70291F30CC00DF
:1022E000183047028A110A16031D78293F30CC00A6
:1022F000193047028A110A16031C80293F30CC008E
:10230000193047028A110A1603188729CD0119309E
:1023100047028A110A16031D8F290130CD001A3099
:1023200047028A110A16031D97290330CD001B307E
:1023300047028A110A16031D9F290730CD001C3061
:1023400047028A110A16031DA7290F30CD001D3040
:1023500047028A110A16031DAF291F30CD001E3017
:1023600047028A110A16031DB7293F30CD001F30DE
:1023700047028A110A16031CBF293F30CD001F30C7
:1023800047028A110A160318C629CE011F304702D8
:102390008A110A16031DCE290130CE0020304702D3
:1023A0008A110A16031DD6290330CE0021304702B8
:1023B0008A110A16031DDE290730CE00223047029B
:1023C0008A110A16031DE6290F30CE00233047027A
:1023D0008A110A16031DEE291F30CE002430470251
:1023E0008A110A16031DF6293F30CE002530470218
:1023F0008A110A16031CFE293F30CE002530470201
:102400008A110A160318052ACF01253047028A11BE
:102410000A16031D0D2A0130CF00263047028A110B
:102420000A16031D152A0330CF00273047028A11F0
:102430000A16031D1D2A0730CF00283047028A11D3
:102440000A16031D252A0F30CF00293047028A11B2
:102450000A16031D2D2A1F30CF002A3047028A1189
:102460000A16031D352A3F30CF002B3047028A1150
:102470000A16031C3D2A3F30CF002B3047028A1139
:102480000A160318442AD0012B3047028A110A1673
:10249000031D4C2A0130D0002C3047028A110A1645
:1024A000031D542A0330D0002D3047028A110A162A
:1024B000031D5C2A0730D0002E3047028A110A160D
:1024C000031D642A0F30D0002F3047028A110A16EC
:1024D000031D6C2A1F30D000303047028A110A16C3
:1024E000031D742A3F30D000313047028A110A168A
:1024F000031C7C2A3F30D000313047028A110A1673
:102500000318832AD101313047028A110A16031DAC
:102510008B2A0130D100323047028A110A16031D7E
:10252000932A0330D100333047028A110A16031D63
:102530009B2A0730D100343047028A110A16031D46
:10254000A32A0F30D100353047028A110A16031D25
:10255000AB2A1F30D100363047028A110A16031DFC
:10256000B32A3F30D100373047028A110A16031CC4
:10257000BB2A3F30D100363047028A110A160318B1
:10258000C22AD201373047028A110A16031DCA2A0D
:102590000130D200383047028A110A16031DD22AB0
:1025A0000330D200393047028A110A16031DDA2A95
:1025B0000730D2003A3047028A110A16031DE22A78
:1025C0000F30D2003B3047028A110A16031DEA2A57
:1025D0001F30D2003C3047028A110A16031DF22A2E
:1025E0003F30D2003D3047028A110A16031CFA2AF6
:1025F0003F30D2000330850087014908880005304C
:102600008A011A204030870087014A088800053077
:102610008A011A204030870087014B088800053066
:102620008A011A204030870087014C088800053055
:102630008A011A204030870087014D088800053044
:102640008A011A204030870087014E088800053033
:102650008A011A204030870087014F088800053022
:102660008A011A2040308700870150088800053011
:102670008A011A2040308700870151088800053000
:102680008A011A20403087008701520888000530EF
:102690008A011A20803087008701880185018A110C
:1026A0000A16061D542B87018A110A16061D5A2B7D
:1026B000013085008A110A16061D602B8A015528F3
:1026C0008A110A16061C662B8A0155288A110A16D9
:1026D000861A6D2B8A110A16772B8A110A16061A8A
:1026E000742B8A110A16772B8A110A167B288A11F5
:1026F0000A16861A7C2BC70A8A110A16061A812B1B
:10270000C7033D3047028A110A16031C882BC701F4
:10271000323003178D00031347088A010C20033061
:10272000A500E8308A011B208A110A16861A9B2B05
:102730008A110A168F2B8A110A16061AA22B8A11E1
:102740000A168F2B8A110A167B288A110A168619F7
:10275000AC2B8A110A16A52B48088A110A16031DEC
:10276000B22BC901013048028A110A16031DBA2B87
:102770000130C900023048028A110A16031DC22B1B
:102780000330C900033048028A110A16031DCA2B00
:102790000730C900043048028A110A16031DD22BE3
:1027A0000F30C900053048028A110A16031DDA2BC2
:1027B0001F30C900063048028A110A16031DE22B99
:1027C0003F30C900073048028A110A16031CEA2B61
:1027D0003F30C900073048028A110A160318F12B4E
:1027E000CA01073048028A110A16031DF92B01306D
:1027F000CA00083048028A110A16031D012C033052
:10280000CA00093048028A110A16031D092C073034
:10281000CA000A3048028A110A16031D112C0F3013
:10282000CA000B3048028A110A16031D192C1F30EA
:10283000CA000C3048028A110A16031D212C3F30B1
:10284000CA000D3048028A110A16031C292C3F3099
:10285000CA000D3048028A110A160318302CCB0129
:102860000D3048028A110A16031D382C0130CB00A6
:102870000E3048028A110A16031D402C0330CB008B
:102880000F3048028A110A16031D482C0730CB006E
:10289000103048028A110A16031D502C0F30CB004D
:1028A000113048028A110A16031D582C1F30CB0024
:1028B000123048028A110A16031D602C3F30CB00EB
:1028C000133048028A110A16031C682C3F30CB00D3
:1028D000133048028A110A1603186F2CCC011330EA
:1028E00048028A110A16031D772C0130CC001430DF
:1028F00048028A110A16031D7F2C0330CC001530C4
:1029000048028A110A16031D872C0730CC001630A6
:1029100048028A110A16031D8F2C0F30CC00173085
:1029200048028A110A16031D972C1F30CC0018305C
:1029300048028A110A16031D9F2C3F30CC00193023
:1029400048028A110A16031CA72C3F30CC0019300C
:1029500048028A110A160318AE2CCD01193048021C
:102960008A110A16031DB62C0130CD001A30480218
:102970008A110A16031DBE2C0330CD001B304802FD
:102980008A110A16031DC62C0730CD001C304802E0
:102990008A110A16031DCE2C0F30CD001D304802BF
:1029A0008A110A16031DD62C1F30CD001E30480296
:1029B0008A110A16031DDE2C3F30CD001F3048025D
:1029C0008A110A16031CE62C3F30CD001F30480246
:1029D0008A110A160318ED2CCE011F3048028A1105
:1029E0000A16031DF52C0130CE00203048028A1152
:1029F0000A16031DFD2C0330CE00213048028A1137
:102A00000A16031D052D0730CE00223048028A1118
:102A10000A16031D0D2D0F30CE00233048028A11F7
:102A20000A16031D152D1F30CE00243048028A11CE
:102A30000A16031D1D2D3F30CE00253048028A1195
:102A40000A16031C252D3F30CE00253048028A117E
:102A50000A1603182C2DCF01253048028A110A16B8
:102A6000031D342D0130CF00263048028A110A168A
:102A7000031D3C2D0330CF00273048028A110A166F
:102A8000031D442D0730CF00283048028A110A1652
:102A9000031D4C2D0F30CF00293048028A110A1631
:102AA000031D542D1F30CF002A3048028A110A1608
:102AB000031D5C2D3F30CF002B3048028A110A16CF
:102AC000031C642D3F30CF002B3048028A110A16B8
:102AD00003186B2DD0012B3048028A110A16031DF2
:102AE000732D0130D0002C3048028A110A16031DC4
:102AF0007B2D0330D0002D3048028A110A16031DA9
:102B0000832D0730D0002E3048028A110A16031D8B
:102B10008B2D0F30D0002F3048028A110A16031D6A
:102B2000932D1F30D000303048028A110A16031D41
:102B30009B2D3F30D000313048028A110A16031C09
:102B4000A32D3F30D000313048028A110A160318F5
:102B5000AA2DD101313048028A110A16031DB22D67
:102B60000130D100323048028A110A16031DBA2DF5
:102B70000330D100333048028A110A16031DC22DDA
:102B80000730D100343048028A110A16031DCA2DBD
:102B90000F30D100353048028A110A16031DD22D9C
:102BA0001F30D100363048028A110A16031DDA2D73
:102BB0003F30D100373048028A110A16031CE22D3B
:102BC0003F30D100373048028A110A160318E92D28
:102BD000D201373048028A110A16031DF12D013047
:102BE000D200383048028A110A16031DF92D03302D
:102BF000D200393048028A110A16031D012E07300F
:102C0000D2003A3048028A110A16031D092E0F30ED
:102C1000D2003B3048028A110A16031D112E1F30C4
:102C2000D2003C3048028A110A16031D192E3F308B
:102C3000D2003D3048028A110A16031C212E3F3073
:102C4000D2000330850087014908870005308A01DA
:102C50001A20403087004A08870005308A011A2070
:102C6000403087004B08870005308A011A20403029
:102C700087004C08870005308A011A204030870001
:102C80004D08870005308A011A20403087004E0821
:102C9000870005308A011A20403087004F088700DE
:102CA00005308A011A20403087005008870005301F
:102CB0008A011A20403087005108870005308A01B8
:102CC0001A20403087005208870005308A011A20F8
:102CD000803087008701880185018A110A16061D48
:102CE000722E87018A110A16061D782E0130850082
:102CF0008A110A16061D7E2E8A0155288A110A1687
:102D0000061C842E8A0155288A110A16061D892E52
:102D100087018A110A16061D8F2E013085008A113F
:102D20000A168618962E8A150A126F2A8A110A1612
:102D3000061D9C2E8A0155288A110A16061CA22EF1
:102D40008A0155288A110A168619A92E8A110A168F
:102D5000E82E8A110A16861AB02E8A110A16BA2E81
:102D60008A110A16061AB72E8A110A16BA2E8A1165
:102D70000A16AC2B8A110A16861ABF2EC80A8A11A7
:102D80000A16061AC42EC8033D3048028A110A16D4
:102D9000031CCB2EC8013C3003178D0003134808D9
:102DA0008A010C200330A500E8308A011B208A111B
:102DB0000A16861ADE2E8A110A16D22E8A110A16D1
:102DC000061AE52E8A110A16D22E8A110A16AC2B83
:102DD0008A110A168619EF2E8A110A16E82E033078
:0E2DE000A500E8308A011B208A110A167B2804
:02400E007A3FF7
:00000001FF
